:0200000480007A
:100000006F00C0006F2080306F20403093000000F0
:10001000130100009301000013020000930200008E
:100020001303000093030000130400009304000076
:10003000130500009305000013060000930600005E
:100040001307000093070000130800009308000046
:100050001309000093090000130A0000930A00002E
:10006000130B0000930B0000130C0000930C000016
:10007000130D0000930D0000130E0000930E0000FE
:10008000130F0000930F00009702000093820201FB
:10009000739052307350447497020000938202F7B9
:1000A0007390523017C100001301C1ECF32240F1EC
:1000B0009392C2003301510073100134EF20101CE1
:1000C000173500001305059D6F20007D832245082C
:1000D0007390121483204500032185008321C500FD
:1000E0000322050183224501032385018323C501E2
:1000F00003240502832445028325C5020326050344
:1001000083264503032785038327C50303280504A6
:1001100083284504032985048329C504032A05058A
:10012000832A4505032B8505832BC505032C05066E
:10013000832C4506032D8506832DC506032E050752
:10014000832E4507032F8507832FC50703258502C7
:100150007300201073110114232211002326310093
:1001600023284100232A5100232C6100232E7100F3
:1001700023208102232291022324A1022326B102FB
:100180002328C102232AD102232CE102232EF102CB
:1001900023200105232211052324210523263105CF
:1001A00023284105232A5105232C6105232E71059F
:1001B00023208107232291072324A1072326B107A7
:1001C0002328C107232AD107232CE107232EF10777
:1001D000F312011423245100F322001023205108AC
:1001E000F322101423225108F3223014232451083F
:1001F000F322201423265108130501006F20803FAD
:1010000000000000000000000000000000000000E0
:1010100000000000000000000000000000000000D0
:1010200000000000000000000000000000000000C0
:1010300000000000000000000000000000000000B0
:081040000000000000000000A8
:10200000B367B500B3E7C70093F73700B306C50061
:10201000638407023386C50093070500637ED502FB
:1020200003C705009385150093871700A38FE7FE6C
:10203000E398C5FE67800000E37ED5FE93070500A8
:1020400003A70500938747009385450023AEE7FE6D
:10205000E3E8D7FE6780000067800000130101FFFE
:10206000B367C500232481002326110093F73700AE
:10207000130405003307C500638207026376E50099
:1020800093F5F50FEFF09FFD8320C10013050400C9
:1020900003248100130101016780000093F5F50F0F
:1020A00093968500B386B60093970601B386F60033
:1020B000E37CE5FC930705009387470023AED7FE3A
:1020C000E3ECE7FE8320C100130504000324810034
:1020D000130101016780000083470500638E07003C
:1020E0009307050003C7170093871700E31C07FE3B
:1020F0003385A7406780000013050000678000005B
:1021000083470500938515001305150003C7F5FFE8
:1021100063880700E386E7FE3385E74067800000B9
:10212000930700006FF05FFFB367B50093F73700C8
:10213000639E07021378C6FF330805016378050321
:10214000930705006F0000019387470093854500C2
:1021500063F8070183A6070003A70500E386E6FEF0
:102160003385A7403306A640138507003386C50094
:102170006F00400103C705008347F5FF93851500F5
:10218000639AE70013051500E396C5FE13050000EA
:10219000678000003385E7406780000093070500F3
:1021A00003C705009387170093851500A38FE7FEEB
:1021B000E31807FE6780000003470500930600024E
:1021C000930705006318D70003C71700938717000C
:1021D000E30CD7FE9306D0026300D7069306B00245
:1021E0006300D70483C607009305000063820604DA
:1021F000130500009387170013172500138606FDAB
:1022000083C607003307A700131717003305E6003E
:10221000E39206FE638005023305A040678000005C
:1022200083C617009305000093871700E39206FC0E
:10223000130500006780000083C617009305100097
:1022400093871700E39606FA130500006FF09FFED0
:10225000834505006380050697F6FFFF938686DABF
:1022600017F6FFFF130606DE03A7060083A7460046
:1022700013880500130515003367F700B70801013F
:1022800063020702130700002320E6009307000003
:102290002322F60003A7060083A746003367F70052
:1022A000E31207FE23A0060123A2160183450500C1
:1022B000E39C05FA6780000097F6FFFF938686D4BB
:1022C00003A7060083A74600130805009358F541AD
:1022D0003367F7006306070217F6FFFF130686D67B
:1022E000130700002320E600930700002322F600D6
:1022F00003A7060083A746003367F700E31207FE33
:1023000023A0060123A216016F000000130101FFA4
:102310001305903423261100EFF01FFA130101FE7C
:102320001306C1001307B101130390006F00800072
:10233000138707009377F500B337F300B307F04036
:1023400093F777029376F50093870703B387F60038
:102350002300F7009396C501135545009307F7FF37
:1023600033E5A60093D54500E314E6FC0345C10020
:10237000230E0100630205069305060097F6FFFF92
:10238000938646C817F6FFFF1306C6CB03A70600C1
:1023900083A7460013080500938515003367F700EF
:1023A000B708010163020702130700002320E600BB
:1023B000930700002322F60003A7060083A7460028
:1023C0003367F700E31207FE03C5050023A00601EB
:1023D00023A21601E31C05FA130101026780000025
:1023E000130101FD9307100037F7FFFF2326F100CB
:1023F0002326110223248102232291022320210378
:10240000232E3101232C4101232A510123240100D1
:10241000B306E500B7E7030063F6F6189359C50065
:1024200093840940174900001309C9BD93972400FC
:10243000B307F90083A707003374E500639607101C
:1024400017670000130747BC032A070063000A1838
:1024500083274A009766000083A6C6BA2320F700A8
:10246000638CD7121306C100930581001305040085
:10247000832A0A00EF0040616310051093D6CA005A
:102480009396A60093E6F60193972400B307F9000C
:1024900013E7060C23A0E70073000412973700002F
:1024A000938747B693993900B387370103A707008D
:1024B0006318071203270A00B705040023A0E700EA
:1024C00003274A0023A2E700F3A50510B707C0FFC2
:1024D000B307F40037160000130704003386C70063
:1024E00003A3070083A8470003A8870003A5C7002C
:1024F0002320670023221701232407012326A70096
:102500009387070113070701E39CC7FC739005102D
:1025100093972400B304F90023A0D400730004129D
:102520000F1000008320C102032481028324410292
:10253000032901028329C101032A8101832A410160
:10254000130101036780000013F707046302070407
:1025500013F70708631207061307F00093E707084D
:10256000639CE50493942400B304990023A0F40031
:10257000730004126FF01FFB83260A00832781007B
:1025800093D6C6009396A600B3E6F6006FF0DFEF91
:1025900093E707046FF01FFD9767000023A407A6C9
:1025A0006FF05FEC1715000013054589EFF05FCA67
:1025B00013053000EFF05FD0171500001305458CB0
:1025C000EFF01FC913053000EFF01FCF1715000003
:1025D0001305858FEFF0DFC713053000EFF0DFCD77
:1025E000171500001305C58FEFF09FC613053000C7
:1025F000EFF09FCC130101FB232481042326110457
:102600002322910423202105232E3103232C41036F
:10261000232A5103232861032326710323248103E2
:10262000232291032320A103232EB10113040500CB
:10263000EF000045631205108325C408930780004E
:102640006380F512930720006380F506938745FFAA
:10265000130710006376F7009307F000639CF520E2
:1026600003258408EFF0DFD7130504000324810459
:102670008320C10483244104032901048329C10365
:10268000032A8103832A4103032B0103832BC10205
:10269000032C8102832C4102032D0102832DC101F1
:1026A000130101056FD09FA20327440893773700D9
:1026B000639E0708EF0780007310300003270700B0
:1026C00083A707006300F70813051004971500009F
:1026D0009385C58497F6FFFF9386C69217F6FFFF92
:1026E0001306469603A7060083A7460013090500B4
:1026F000938515003367F700B709010163020702EC
:10270000930700002320F60013080000232206018F
:1027100003A7060083A746003367F700E31207FE0E
:1027200003C5050023A0260123A23601E31C05FAF8
:1027300013053000EFF05FB813050400EFD01F99C8
:102740006FF09FEF13051000EFF01FB71715000093
:1027500013050586EFF0DFAF13053000EFF0DFB5AE
:102760008327840237190000973A0000938A8A89E8
:102770002326F100174D0000130DCD88B70C04007F
:10278000370CC0FF176A0000130ACA87976B000056
:10279000938B8B8737FB03009357C90093993700BE
:1027A00033873A0103270700630C07089387074024
:1027B00093972700B307FD0083A4070093F7040451
:1027C0006380070AF3AD0C1033048901371600004B
:1027D0009305040013050900EFF01F956304050439
:1027E00093F404086380040AB71600001307090075
:1027F00093070400B306D900032807000325470008
:10280000832587000326C70023A0070123A2A70072
:1028100023A4B70023A6C700130707019387070166
:10282000E31CD7FCB3873A0173900D1003270A000D
:1028300023A00700630007022322F7002320FA00E9
:10284000B71700003309F900E31869F50325C10043
:10285000EFF09FA62320FA0023A0FB006FF05FFE9D
:10286000170500001305456EEFF09F9E130530001D
:10287000EFF09FA4170500001305C575EFF05F9DED
:102880006FF01FEB170500001305456FEFF05F9C1D
:1028900013053000EFF05FA2F32740F163960716AF
:1028A00017460000130606769357C600130101F67B
:1028B0009397A700232E1108232C81089735000039
:1028C0009385457493E7170023A0F500B707002010
:1028D00093D6C500370700809387F70C232EF6FEAA
:1028E000B3E7E60073900718F3260018639ED71627
:1028F000130405001347F7FF9307F0019702000048
:1029000093824201F39252307310073B7390073A5F
:102910007390523097E7BF7F938707847390571067
:10292000F3270034B708C07FB387170173900714EB
:10293000B7B700009387071073902730B7E70100FF
:102940009387076073900730735040309737C07F8C
:102950009387C78A175700002328F76A9737C07FE5
:102960009387C7A817570000232EF768370308007E
:102970001737000013078788173E0000130E8EA735
:102980009307B002930500001303F30393888800B4
:102990001396F50193D61700B366D6003386670009
:1029A000B3C7F600330817011316C60093975700F4
:1029B0002320C7002322070193F70702130787008C
:1029C000B3E7F60093D51500E314EEFC13060009F7
:1029D00093050000130501009737000023AA07A004
:1029E000EFF0CFE7B70700803304F40013050100D0
:1029F00023228108EFD08FED8320C10903248109B0
:102A00001301010A67800000B787120D370608001E
:102A10009387F7C7130700001306C6FF3708008027
:102A2000370500406F00C0022FA006009315F70184
:102A300093D61700B3E6D500B3C7D7009397E70145
:102A4000B375F500135717009387060033E7E500C9
:102A5000B3F6C70093F51700B3860601E39605FCAD
:102A600003A006006FF09FFC1705000013054559F1
:102A7000EFF00FFE13053000EFF01F8467800000B9
:102A80001305000067800000130500006780000048
:102A900073103000930120001715000013058556B0
:102AA0000730050087308500073105018326850141
:102AB0000323C501532510A293030000F315100052
:102AC00013060000631CD534631A73346398C5344D
:102AD00093013000171500001305C5540730050099
:102AE0008730850007310501832685010323C50151
:102AF000530510A293030000F31510001306000005
:102B0000631ED530631C7330639AC5309301400057
:102B100017150000130505530730050087308500A1
:102B200007310501832685010323C501531510A232
:102B300093030000F3151000130600006310D52E58
:102B4000631E732C639CC52C930150001715000065
:102B50001305455107300500873085000731050111
:102B6000832685010323C501532510A2930300008A
:102B7000F3151000130600006312D52A6310732AA0
:102B8000639EC52893016000171500001305854F4B
:102B90000730050087308500073105018326850150
:102BA0000323C501530510A293030000F315100081
:102BB000130600006314D526631273266390C5269E
:102BC00093017000171500001305C54D073005006F
:102BD0008730850007310501832685010323C50160
:102BE000531510A293030000F31510001306000004
:102BF0006316D522631473226392C5229301800069
:102C0000171500001305054C0730050087308500B7
:102C100007310501832685010323C501532510A231
:102C200093030000F3151000130600006318D51E6F
:102C30006316731E6394C51E930190001715000060
:102C40001305454A07300500873085000731050127
:102C5000832685010323C501532510A29303000099
:102C6000F315100013060000631AD51A6318731ABF
:102C70006396C51A9301A000171500001305854837
:102C8000073005008730850007310501832685015F
:102C90000323C501532510A293030000F315100070
:102CA00013060001631CD516631A73166398C516C4
:102CB0009301B000171500001305C5460730050045
:102CC0008730850007310501832685010323C5016F
:102CD000531510A293030000F31510001306000112
:102CE000631ED512631C7312639AC5129301C00050
:102CF00017150000130505450730050087308500CE
:102D000007310501832685010323C501531510A250
:102D100093030000F3151000130600016310D51093
:102D2000631E730E639CC50E9301D000171500003F
:102D3000130545430730050087308500073105013D
:102D4000832685010323C501531510A293030000B8
:102D5000F3151000130600016312D50C6310730CF9
:102D6000639EC50A9301E000171500001305854115
:102D7000073005008730850007310501832685016E
:102D80000323C501530510A293030000F31510009F
:102D9000130600016314D508631273086390C50815
:102DA0009301F000171500001305C53F073005001B
:102DB0008730850007310501832685010323C5017E
:102DC000530510A293030000F31510001306000131
:102DD0006316D504631473046392C5049301000160
:102DE000171500001305053E0730050087308500E4
:102DF00007310501832685010323C501530510A270
:102E000093030000F3151000130600016318D500AA
:102E1000631673006394C500631A300013951100A4
:102E20006300050013651500730000001305100012
:082E300073000000731000C0E4
:102E3800417373657274696F6E206661696C65644D
:102E48003A2061646472203E3D202831554C203C74
:102E58003C203132292026262061646472203C20DF
:102E68003633202A202831554C203C3C2031322949
:102E78000A000000417373657274696F6E206661A1
:102E8800696C65643A20212870745B315D5B61640C
:102E980064722F2831554C203C3C203132295D206A
:102EA8002620307830383029202626206361757333
:102EB80065203D3D203078660A0000004173736547
:102EC8007274696F6E206661696C65643A206E6F12
:102ED80064650A00417373657274696F6E20666178
:102EE800696C65643A20757365725F6D61707069AD
:102EF8006E675B616464722F2831554C203C3C201E
:102F08003132295D2E61646472203D3D20300A0013
:102F1800417373657274696F6E206661696C65646C
:102F28003A202122696C6C6567616C20696E737444
:102F380072756374696F6E220A00000041737365CD
:102F48007274696F6E206661696C65643A2070748A
:102F58005B315D5B616464722F2831554C203C3CC9
:102F6800203132295D20262030783034300A0000A4
:102F7800417373657274696F6E206661696C65640C
:102F88003A2070745B315D5B616464722F2831553F
:102F98004C203C3C203132295D20262030783038C6
:102FA800300A0000417373657274696F6E20666140
:102FB800696C65643A2074662D3E6570632025202F
:102FC80034203D3D20300A00417373657274696F87
:102FD8006E206661696C65643A202122756E657899
:102FE80070656374656420657863657074696F6E75
:102FF800220A0000417373657274696F6E206661FE
:10300800696C65643A202122756E737570706F72F1
:103018007465642073617470206D6F6465220A00A2
:10400000C3F5285C8FC2F5BFC3F5285C8FC2F5BF2E
:10401000000000000000000001000000000000009F
:10402000C3F5285C8FC2F5BFC3F5285C8FC2F5BF0E
:10403000000000000000000001000000000000007F
:10404000C3F5285C8FC2F5BFC3F5285C8FC2F5BFEE
:104050000000000000000000000000000000000060
:10406000EC51B81E85EBF5BFC3F5285C8FC2F5BFD8
:104070000000000000000000000000000000000040
:10408000EC51B81E85EBF5BFC3F5285C8FC2F5BFB8
:10409000000000000000000001000000000000001F
:1040A000EC51B81E85EBF5BFC3F5285C8FC2F5BF98
:1040B00000000000000000000100000000000000FF
:1040C000FFFFFFFFFFFFFF7F000000000000000078
:1040D00000000000000000000000000000000000E0
:1040E000FFFFFFFFFFFFFF7FFFFFFFFFFFFFFF7FE0
:1040F00000000000000000000000000000000000C0
:10410000010000000000F07F00000000000000003F
:10411000000000000000000000000000000000009F
:10412000FFFFFFFFFFFFFF7F000000000000000017
:10413000000000000000000000000000000000007F
:10414000FFFFFFFFFFFFFF7FFFFFFFFFFFFFFF7F7F
:10415000000000000000000000000000000000005F
:10416000010000000000F07F0000000000000000DF
:10417000000000000000000000000000000000003F
:10418000FFFFFFFFFFFFFF7F0000000000000000B7
:10419000000000000000000000000000000000001F
:1041A000FFFFFFFFFFFFFF7FFFFFFFFFFFFFFF7F1F
:1041B00000000000000000000000000000000000FF
:1041C000010000000000F07F00000000000000007F
:1041D00000000000000000000000000000000000DF
:040000058000000077
:00000001FF
